:100000002CC054C053C052C051C051C04FC04EC08C
:100010004DC04CC04BC04AC049C048C047C000009A
:1000200000000000000000000000000023456C9864
:10003000C9FF040714233764A0FFFFFFFFFFFFFF82
:10004000FFFFFFFFFF000000000000000000234052
:100050005F7AB4FFFFFFFFFFFF0011241FBECFE553
:10006000D2E0DEBFCDBF20E0A0E6B0E001C01D922F
:10007000A738B207E1F7E2E6F0E085E5808781E0A6
:1000800083831482128287E086831182ADE6B0E01A
:100090008EEF15968C9315978DEF17968C9311868E
:1000A00088E58287612C712C86D0C4C0A9CF1895B1
:1000B00025B7277E25BF29B7226029BF21E022BFAF
:1000C000019728F020E188952150E9F7F9CF0895AC
:1000D00088EE93E0EDCF8CE287B986EC86B9369A4C
:1000E0003699FECF8FEF809360000895369A369947
:1000F000FECF95B18091600089270895811104C0D9
:100100001BBC19BC18BC0895815090E0FC01E25E54
:10011000FF4FE491EBBDFC01EE5CFF4FE491E9BDC4
:10012000FC01EA5BFF4F849188BD08950F931F93F4
:10013000CF93C82F8B01CC2369F085E0DFDFC801A6
:10014000B7DF1BBC19BC18BCC801B2DFC801B0DFE7
:10015000C150F1CFCF911F910F910895CF93DF93AD
:10016000D82F64E170E08AE0E1DF84EF91E0A0DF66
:100170008D2F64E653D0CAE06C2F50D0892F68ECE5
:1001800070E0D4DFA5DF8D2F6C2F48D0D92F46D05B
:10019000892F68EC70E0CADF9BDF68EC70E08D2F80
:1001A000C5DF96DF64E170E08AE0C0DF84EF91E0B4
:1001B000DF91CF917DCF83EA87B986EC86B93699F6
:1001C000FECF369A3699FECF85B18FE384BBBB9ABA
:1001D000C39AB99AB89ABC9A81E08ABD83BF9AB58E
:1001E00090629ABD9AB590689ABD9FEF9DBD80BF01
:1001F00080E68CBD97B328B3892F90E080959095C9
:100200008B7F822B88BB85B7806285BF789463DF44
:100210008CE291E04DDF6ADFA1DFFACF991B79E034
:1002200004C0991F961708F0961B881F7A95C9F786
:0802300080950895F894FFCFBA
:00000001FF
